:0200000480007A
:100000006F000005732F2034930F80006308FF03F7
:10001000930F90006304FF03930FB0006300FF038E
:10002000130F000063040F0067000F00732F2034CC
:1000300063540F006F00400093E19153171F0000BD
:1000400023223FFC171F000023200FFC6FF01FFF2F
:100050009300000013010000930100001302000050
:100060009302000013030000930300001304000038
:100070009304000013050000930500001306000020
:100080009306000013070000930700001308000008
:10009000930800001309000093090000130A0000F0
:1000A000930A0000130B0000930B0000130C0000D8
:1000B000930C0000130D0000930D0000130E0000C0
:1000C000930E0000130F0000930F0000732540F102
:1000D0006310050097020000938202017390523072
:1000E000735044749702000093820201739052305F
:1000F00073500018970200009382020273905230EE
:10010000B70200809382F2FF7390023B9302F001EA
:100110007390023A7350403097020000938242017C
:100120007390523073502030735030309301000080
:1001300097020000938242ED739052301305100035
:100140001315F501634C05000F00F00F930110002B
:100150009308D0051305000073000000930200000F
:10016000638A020073905210B7B20000938292101B
:100170007390223073500030970200009382420146
:1001800073901234732540F17300203093012000E6
:10019000930000001301000033A720029303000026
:1001A000631A774A93013000930010001301100086
:1001B00033A7200293030000631E77489301400099
:1001C000930030001301700033A720029303000056
:1001D0006312774893015000930000003781FFFFBE
:1001E00033A7200293030000631677469301600053
:1001F000B70000801301000033A720029303000022
:10020000631A774493017000B70000803781FFFFC5
:1002100033A72002B7430080631E77429301E001B9
:10022000B7B0AAAA9380B0AA370103001301D1E79F
:1002300033A72002B703FFFF93831308631C7740A3
:100240009301F001B70003009380D0E737B1AAAA69
:100250001301B1AA33A72002B70302009383E3EF8F
:10026000631A773E93010002B70000FF370100FFD9
:1002700033A72002B70301FF631E773C93011002EE
:100280009300F0FF1301F0FF33A720029303F0FF68
:100290006312773C930120029300F0FF13011000DA
:1002A00033A720029303F0FF6316773A93013002DD
:1002B000930010001301F0FF33A720029303000006
:1002C000631A773893018000B700D0003701B0007F
:1002D000B3A02002B7930000938303F0639C7036B1
:1002E00093019000B700E0003701B00033A1200275
:1002F000B7A30000938303A0631E71349301A00091
:10030000B700D000B3A01002B7B3000093830390EE
:10031000639270349301B00013020000B700D00064
:100320003701B00033A720021303070013021200A5
:1003300093022000E31452FEB7930000938303F06E
:10034000631A73309301C00013020000B700E0008D
:100350003701B00033A72002130000001303070089
:100360001302120093022000E31252FEB7A3000012
:10037000938303A06310732E9301D0001302000037
:10038000B700F0003701B00033A7200213000000CF
:100390001300000013030700130212009302200051
:1003A000E31052FEB7A30000938303506314732A33
:1003B0009301E00013020000B700D0003701B00045
:1003C00033A720021302120093022000E31652FE0C
:1003D000B7930000938303F0631E77269301F00028
:1003E00013020000B700E0003701B0001300000066
:1003F00033A720021302120093022000E31452FEDE
:10040000B7A30000938303A0631677249301000130
:1004100013020000B700F0003701B0001300000025
:100420001300000033A720021302120093022000E1
:10043000E31252FEB7A3000093830350631C77209E
:100440009301100113020000B700D0001300000058
:100450003701B00033A720021302120093022000DC
:10046000E31452FEB7930000938303F06314771EE6
:100470009301200113020000B700E0001300000008
:100480003701B0001300000033A72002130212004E
:1004900093022000E31252FEB7A30000938303A04F
:1004A000631A771A9301300113020000B700F000BD
:1004B00013000000130000003701B00033A7200232
:1004C0001302120093022000E31252FEB7A30000B1
:1004D00093830350631077189301400113020000C7
:1004E0003701B000B700D00033A72002130212007A
:1004F00093022000E31652FEB7930000938303F0AB
:10050000631A771493015001130200003701B00001
:10051000B700E0001300000033A72002130212000E
:1005200093022000E31452FEB7A30000938303A0BC
:100530006312771293016001130200003701B000CB
:10054000B700F000130000001300000033A72002E2
:100550001302120093022000E31252FEB7A3000020
:10056000938303506318770E930170011302000008
:100570003701B00013000000B700D00033A72002FD
:100580001302120093022000E31452FEB7930000FE
:10059000938303F06310770C930180011302000032
:1005A0003701B00013000000B700E00013000000A6
:1005B00033A720021302120093022000E31252FE1E
:1005C000B7A30000938303A06316770893019001FB
:1005D000130200003701B0001300000013000000F8
:1005E000B700F00033A7200213021200930220008C
:1005F000E31252FEB7A3000093830350631C7704F9
:100600009301A001B700007C332110029303000086
:10061000631271049301B001B700008033A100029E
:1006200093030000631871029301C001B32000021C
:1006300093030000639070029301D001B700100291
:100640003701200233A020029303000063147000DE
:10065000631030020F00F00F6380010093911100CE
:1006600093E111009308D005138501007300000089
:100670000F00F00F930110009308D0051305000040
:1006800073000000731000C00000000000000000B4
:10069000000000000000000000000000000000005A
:1006A000000000000000000000000000000000004A
:0C06B0000000000000000000000000003E
:1010000000000000000000000000000000000000E0
:1010100000000000000000000000000000000000D0
:1010200000000000000000000000000000000000C0
:1010300000000000000000000000000000000000B0
:081040000000000000000000A8
:040000058000000077
:00000001FF
